:020000040000FA
:10000000831603138101402C8B138B1B0428AD0036
:10001000030EAE0083010A08AF008A0183130408AF
:10002000B0008B1824288C1A16287A281A08AA00DF
:100030008C1E1D281A08AB002817271483160313DB
:100040008C12831203137A28281C4A283208073C92
:10005000031C3028331C051233180516B30C7828FE
:100060003208083C031C3928A81C0512A8180516DC
:1000700078283208093C031C43288316031305160D
:1000800083120313782832080B3C031C7828B20132
:1000900028107928B208031D5028051A75287828D9
:1000A0003208083C031C5C28051EB313051AB3175D
:1000B00003197828B30C78283208093C031C6128FE
:1000C0007828051E752828196E28A717831603138C
:1000D00006108312031306100B127628230833022E
:1000E000031D75282811B2017928B301B2017928BE
:1000F000B20A8B10300884002F088A002E0E83006D
:10010000AD0E2D0E09003308B400F03C031D8B2802
:10011000A714A711252BA71CA92AA7103308123C46
:10012000031995283308593C031927113308583C03
:10013000031DBA28271EAB282712ED30B300762105
:100140005D21FA30832135113508B30076215D2118
:10015000FA308321252B2716ED30B30076215D215F
:10016000FA30832135153508B30076215D21FA3048
:100170008321252B3308113C031DC028A712662BB1
:0C0180003308143C031D252B27139D2B76
:10020000A000810183160313C03081050800A000FF
:10021000810183160313C0308105013081048312EC
:1002200003130B110B1D1229A00B11290800A200AA
:10023000E1308605220D1E39860408002816212982
:100240002812A3003A21281E86172308230E1721FF
:100250003121230817213121E13086058613061349
:10026000080086160000861208001830A200A20BB3
:10027000372908008613A815831603131E30860439
:10028000831203130617000086163521061EA811D7
:10029000861235213121A819442906138316031328
:1002A000E130860583120313080083160313981C9C
:1002B000572983120313990008000B1283160313A6
:1002C0000610051283120313061005122030A00039
:1002D000A00B6829B20183160313061483120313BB
:1002E00028148B100B16281873290800A200083058
:1002F000A300A4012218A40AA20CA30B7A29A81017
:10030000241CA8140800A300281528198529080012
:100310002A08AC009C21281F96292B08AC009C21A0
:100320002813981C962918121811181683160313EF
:100330008C168312031308002C08083C031DAA29FD
:1003400036080319BF29B603360880381E2120302D
:100350002021BF293608273C0318B029A812C12143
:10036000360880381E212C080D3C031CBC29031DB7
:10037000BF29A812C121BF292C082021B60A2710A5
:1003800008002830A81ACF29B60080301E2120305E
:100390002021B60BC72980301E21B6010800B70006
:1003A000C0301E2120302021B70BD229C0301E21A1
:0403B000B701080089
:100460008207003439340034353433343134323493
:1004700032340034303438343634343409347E3451
:10048000003400342F2B2D2B0034312B71343134B8
:100490000034003400347A347334613477343234C5
:1004A00000340034633478346434653434343334A1
:1004B0000034003420347634663474347234353485
:1004C000003400346E34623468346734793436343E
:1004D0000034003400346D346A34753437343834C1
:1004E000003400342C346B3469346F343034393494
:1004F000003400342E343F346C343B3470342D34AB
:10050000003400340034273400345B342B3400349E
:10051000003400342D2B1E2B5D3400347C34003429
:10052000003400343C3430342E34323435343634F4
:1005300038340034003431342B3433342D342A34FD
:10054000393400340834003400343134373434342E
:100550003734A71DBB2AA71ABB2A271BBB2A33087F
:100560004A3C031DB62A2F30B300EF2A33085A3C09
:100570000318BB2A252B3308613C0318D12A0E30FF
:10058000B3023308613C031CC82A1930B307D12ACF
:100590003308773C0318D12A3308D23C0319A71536
:1005A000252B02308A0033083022B300B308031928
:1005B000252BA71A492B271B372B3308603C031820
:1005C000B62B33087A3C031CB62B3308271AEB2AC8
:1005D000271DEF2AED2A2719EF2AE03EB300330842
:1005E00055213308083C031D032B37080319252B1D
:1005F000B7033708403E8038A5001E212030202157
:1006000025081E21252B3308093C031D102B370814
:10061000263C031C0E2B20302021B70A2030B300CB
:100620003708273C0318162BA816C1213708403E6F
:1006300080381E2133082021B70A252BA816C12196
:100640000D3055210A30552100348316031306144A
:1006500083120313A7130B16080027150034A716DF
:10066000322B2717B801B901BA01BB010034330896
:10067000403C0318492B3308463C031C412BB3165E
:10068000512B3308603C0318492B3308663C031890
:10069000512B3308293C0318252B3308393C031C04
:1006A000252BB808031D582BB80A3308B900252B91
:1006B000380B5E2BB80A3308BA00252B3808023CE9
:1006C000031D252BB80A3308BB00252BB8080319D6
:1006D000252B3030B902BA02BB02B803031D732BBD
:1006E0003908B3008D2BB803031D7D2B03308A001E
:1006F00039088F233A07B3008D2B3908023C031CBD
:10070000252B03308A0039080A3E8F23B9003A08A6
:100710008F23B9073B083907B300B801EF2A8207D6
:1007200000340A3414341E34283432343C34463411
:1007300050345A3400346434C834B8080319252BB3
:100740003030B902BA02B91EA72B2730B902BA1E3F
:10075000AB2B2730BA02B803031DB12B3908B30005
:10076000B42B390E3A04B300B801EF2A271DEF2A43
:1007700033080D3C0318EF2A3408613C031CEF2AB0
:1007800034083C3C0318C72B3D30B402D02B34084E
:10079000243C0318CE2B2330B402D02B0430B407F2
:1007A00003308A003408D623B300EF2A82072634A8
:1007B0002A34243423343C340034003400342934C3
:1007C0002834003425343E342F3400343A34003495
:1007D0005F3460345E340034223400347B343D3482
:1007E000003421340034003400347D3400345C346F
:0807F0000034403400343E34B3
:1008800002309F00831203138316031318151930C7
:100890009900831203139817831603138C16981666
:1008A000831203130B171816831603130614051669
:1008B0000113831203130B16F8308B058C018D0185
:1008C0008B170230B500B201A701A80183160313EC
:1008D0000130860583120313861206138613E13056
:1008E000860504300721033017213121013007210B
:1008F0000830172131210130072102301721312121
:100900000130072128301E210C301E2101301E210C
:10091000083007212830B600B7012730A500043081
:100920008A002508273CC224A6005521260820213C
:10093000A50B8F2C0D3055210A3055210A30552139
:10094000FF30B30076215D21ED30B30076215D21CB
:10095000FA3083213508B30076215D21FA308321F6
:10096000ED30B30076215D21FA308321351435084E
:10097000B30076215D21FA308321A71B832027183D
:100980008821BD2C8207503449344334203431341B
:1009900036344634373437342034413454342034F8
:1009A0004B346534793462346F3461347234643476
:1009B00020344434653463346F34643465347234C1
:1009C000203463346F346E346E346534633474347D
:0409D00065346434F2
:02400E00F23F7F
:00000001FF
